:020000040000FA
:06000000E2EF27F0120000
:06002A000200545000002A
:100030006700000050000000525000002601000040
:0400400002000000BA
:0C004400D9CFE6FFE1CFD9FF83E941E806
:100050008A84080EE66E350EE66E3AEC27F042E929
:10006000036A080E035C10E203500024E96E000EE0
:100070000120EA6EEFCFE6FF360E0324E66E3AEC7F
:1000800027F042E9032AEDD7E66A8DEC26F041E934
:100090008A9442E9E7CFD9FF1200D9CFE6FFE1CF3A
:1000A000D9FF85E942E8070E0001015D03E0090E72
:1000B000015D15E100EB13F101EB14F102EB15F119
:1000C00003EB16F101011351066E06EBE6FF430E3A
:1000D000E66E3AEC27F042E906EB3CF21DD000EB6D
:1000E00013F101EB14F102EB15F103EB16F1070E1E
:1000F00001011317146B156B166B1351066E065026
:10010000200DF350066E06EBE6FF420EE66E3AEC6B
:1001100027F042E906EB3CF28A84080EE66E450EB3
:10012000E66E3AEC27F042E9300EE66E460EE66ED9
:100130003AEC27F042E9010E056E080E055C09E273
:10014000E66A460E0524E66E3AEC27F042E9052AF7
:10015000F4D7010EE66E8DEC26F041E98A9443E96E
:10016000E7CFD9FF1200D9CFE6FFE1CFD9FF81E970
:1001700042E88A84080EE66E350EE66E3AEC27F009
:1001800042E9016A080E015C11E20150F76ADE0FD4
:10019000F66E4F0EF7220800F5CFE6FF360E01246B
:1001A000E66E3AEC27F042E9012AECD7E66A8DECDC
:1001B00026F041E98A94010EE66E68DB41E9026EA1
:1001C000050E025C09E07F0E00010A5D05E0210ECC
:1001D0000C5D02E0000E02D00D0E00D043E9E7CF27
:1001E000D9FF1200D9CFE6FFE1CFD9FF82E943E87A
:1001F000005007E07F0E026E840E036EBC0E046E8C
:1002000006D07E0E026E840E036EBC0E046EE66A8D
:10021000E66AE66AFC0EE66E02EBE6FF03EBE6FF3B
:1002200004EBE6FF7F0EE66EE668E66860EC1BF026
:100230004AE944E9E7CFD9FF1200D9CFE6FFE1CF81
:10024000D9FF82E941E800EBE6FFCCDF41E9FB0E94
:10025000E66E310EE66E3AEC27F042E9E00EE66E0D
:10026000320EE66E3AEC27F042E9FC0EE66E410EE5
:10027000E66E3AEC27F042E9E66A420EE66E3AECA8
:1002800027F042E9E668200EE66E3AEC27F042E9F4
:10029000E66A210EE66E3AEC27F042E9FD0EE66EC4
:1002A000E66A3AEC27F042E9E66A010EE66E3AECBD
:1002B00027F042E9240EE66E600EE66E3AEC27F077
:1002C00042E9E668240EE66E3AEC27F042E9E66879
:1002D000250EE66E3AEC27F042E9E668090EE66E76
:1002E0003AEC27F042E9E668110EE66E3AEC27F0A8
:1002F00042E9E668150EE66E3AEC27F042E9E66858
:10030000190EE66E3AEC27F042E9200EE66E700E0A
:10031000E66E3AEC27F042E9E66AAEEC27F041E9F6
:10032000C0EC27F0026EE00E021402E00D0E10D0B9
:100330001ADF026E02500AE10001038103950050AA
:1003400002E0060E01D0080E0001016F025000D03D
:1003500042E9E7CFD9FF1200D9CFE6FFE1CFD9FFBD
:1003600082E941E800EBE6FF3DDF41E9C60EE66EBB
:10037000310EE66E3AEC27F042E9CB0EE66E320E15
:10038000E66E3AEC27F042E9330EE66EE66E3AECA2
:1003900027F042E9F10EE66E340EE66E3AEC27F0F5
:1003A00042E9C60EE66E410EE66E3AEC27F042E9EF
:1003B000EB0EE66E420EE66E3AEC27F042E9E66A94
:1003C000430EE66E3AEC27F042E9F10EE66E440E7B
:1003D000E66E3AEC27F042E9E668200EE66E3AEC6B
:1003E00027F042E9E30EE66E210EE66E3AEC27F0C6
:1003F00042E9E668220EE66E3AEC27F042E9E66A48
:10040000230EE66E3AEC27F042E9C60EE66EE66A87
:100410003AEC27F042E9CA0EE66E010EE66E3AECBF
:1004200027F042E9F10EE66E020EE66E3AEC27F096
:1004300042E9E66A030EE66E3AEC27F042E9440E22
:10044000E66E600EE66E3AEC27F042E9E668240EAE
:10045000E66E3AEC27F042E9E668250EE66E3AECE5
:1004600027F042E9E668090EE66E3AEC27F042E929
:10047000E668110EE66E3AEC27F042E9E668150EE2
:10048000E66E3AEC27F042E9E668190EE66E3AECC1
:1004900027F042E9200EE66E700EE66E3AEC27F089
:1004A00042E9E66AAEEC27F041E9C0EC27F0026EC3
:1004B000E00E021402E00D0E10D055DE026E025066
:1004C0000AE1000103810385005002E0070E01D01C
:1004D000090E0001016F025000D042E9E7CFD9FFB9
:1004E0001200D9CFE6FFE1CFD9FF87E941E800014B
:1004F00000A340D000010351040B01E0010EE66EA1
:10050000150EE66E000EE66E00EBE6FF01EBE6FF71
:1005100002EBE6FF03EBE6FF24EC1DF047E9010FD9
:10052000076E680EE66E2F0EE66E150EE66E000E76
:10053000E66E28EC1FF044E907500101146B150F1B
:10054000136F000E142313C1E6FF14C1E6FF04EB82
:10055000E9FF05EBEAFFEFCFE6FF0428156F000E79
:100560000520166F15C1E6FF16C1E6FFF4EC1CF07E
:1005700045E919D0150EE66E000EE66E0428E96E08
:10058000000E0520EA6EEFCFE6FF020E0101042403
:10059000136F000E0520146F13C1E6FF14C1E6FFB0
:1005A000F4EC1CF045E9150EE66E000EE66E27EC45
:1005B0001BF042E942E9E7CFD9FF1200D9CFE6FFAD
:1005C000E1CFD9FF87E943E8000100A340D0000153
:1005D0000351040B01E0010EE66E150EE66E000EEF
:1005E000E66E00EBE6FF01EBE6FF02EBE6FF03EB56
:1005F000E6FF24EC1DF047E9010F076E680EE66E7A
:100600002F0EE66E150EE66E000EE66E28EC1FF05D
:1006100044E907500101146B150F136F000E1423EA
:1006200013C1E6FF14C1E6FF04EBE9FF05EBEAFFA7
:10063000EFCFE6FF0428156F000E0520166F15C1D9
:10064000E6FF16C1E6FFF4EC1CF045E953D0020EBC
:100650000424E96E000E0520EA6EEF50086E096A68
:100660000428E96E000E0520EA6EEF500F0B010121
:10067000136F13C114F1136B1351081214510912A3
:1006800000010351040B01E0010EE66E150EE66E4B
:10069000000EE66E08EBE6FF09EBE6FFE66AE66AA7
:1006A00024EC1DF047E9150EE66E000EE66E27EC11
:1006B0001BF042E9E60EF66E4F0EF76E0800F5CF1E
:1006C00015F000013A0E166F200E176F180EE66E29
:1006D000000EE66E060EE66E030E01010424136F93
:1006E000000E0520146F13C1E6FF14C1E6FFF4EC01
:1006F0001CF045E9150EE66E000EE66E27EC1BF0C9
:1007000042E944E9E7CFD9FF1200D9CFE6FFE1CFB4
:10071000D9FF87E941E8000100A340D0000103515F
:10072000040B01E0010EE66E150EE66E000EE66E9D
:1007300000EBE6FF01EBE6FF02EBE6FF03EBE6FF73
:1007400024EC1DF047E9010F076E680EE66E2F0ED0
:10075000E66E150EE66E000EE66E28EC1FF044E91C
:1007600007500101146B150F136F000E142313C1F2
:10077000E6FF14C1E6FF04EBE9FF05EBEAFFEFCF6C
:10078000E6FF0428156F000E0520166F15C1E6FF61
:1007900016C1E6FFF4EC1CF045E92AD00428E96E06
:1007A000000E0520EA6EEF500F0B076E0750F76A38
:1007B000E60FF66E4F0EF7220800F5CF15F0000198
:1007C0003A0E166F200E176F180EE66E000EE66ECC
:1007D000070EE66E020E01010424136F000E0520C1
:1007E000146F13C1E6FF14C1E6FFF4EC1CF045E9F9
:1007F000150EE66E000EE66E27EC1BF042E942E9AC
:10080000E7CFD9FF1200D9CFE6FFE1CFD9FF83E9C7
:1008100041E800EBE9FF01EBEAFFEF50080804E0D4
:10082000000EF36EF46A2ED00028E96E000E01204F
:10083000EA6EEF50F00BE8380F0B036E030E035C0B
:1008400004E3000EF36EF46A1DD0035017E1002894
:10085000E96E000E0120EA6EEF50070804E2000E78
:10086000F36EF46A0FD00028E96E000E0120EA6EE4
:10087000EF5004E1000EF36EF46A04D0010EF36E43
:10088000F46A00D042E9E7CFD9FF1200D9CFE6FFE2
:10089000E1CFD9FF82E94AE800010251066EF294E5
:1008A0000650AE0802E2AE0E066E06500101136F4E
:1008B000146B770E1403F3CF14F113511427770E32
:1008C0001303F3CF13F1F4501427FF0ED8801357FE
:1008D000145714C113F1146B1351076E07EBD7FFB4
:1008E0000650136F146B770E1403F3CF14F11351EA
:1008F0001427770E1303F3CF13F1F4501427FF0ED0
:10090000D880135714571351086E08EBD6FF000E0A
:10091000046E020E056E096AF2B479D082B2FCD779
:100920008A8273EC27F0030B0A6E020E0A1402E0AF
:10093000010E01D0000E0B6E01010428136F000E92
:100940000520146F13C1E6FF14C1E6FF04EBE6FFB8
:1009500005EBE6FF090E0424156F000E0520166F47
:1009600015C1E6FF16C1E6FF0BEBE6FFEEEC21F04A
:1009700047E98A9204EBE6FF05EBE6FF44DF42E934
:10098000F3CF13F1F4CF14F101011351141101E16C
:10099000C3D7005002E0080EA3D00428E96E000E71
:1009A0000520EA6EEF50F00BE8380F0B020A1BE04F
:1009B000030A04E0010A01E01BD01AD0090E042446
:1009C000026E000E0520036E02EBE9FF03EBEAFF67
:1009D000EECFE6FFEECFE6FFEECFE6FFEECFE6FF8F
:1009E0004DEC00F044E907EBD7FF08EBD6FF00D051
:1009F0000D0E09260426000E0522F40EF36EF46A8D
:100A00000950F35C000EF45801E201D085D704EBE5
:100A1000E9FF05EBEAFFEF6A000E046E020E056EB9
:100A200004EBE9FF05EBEAFFEF5054E0090E042464
:100A3000026E000E0520036E0428E96E000E0520EC
:100A4000EA6EEF50F00BE8380F0B020A2BE0030AB6
:100A500016E0010A01E039D002EBE9FF03EBEAFFFF
:100A6000EECFE6FFEECFE6FFEECFE6FFEECFE6FFFE
:100A700004EBE6FF05EBE6FF34DD46E926D002EBAA
:100A8000E9FF03EBEAFFEECFE6FFEECFE6FFEECFA6
:100A9000E6FFEECFE6FF04EBE6FF05EBE6FF8EDDBB
:100AA00046E913D002EBE9FF03EBEAFFEECFE6FFE6
:100AB000EECFE6FFEECFE6FFEECFE6FF04EBE6FF7C
:100AC00005EBE6FF22DE46E900D00D0E0426000EFF
:100AD0000522A6D7095002E0080E01D0050E00D06D
:100AE0004BE9E7CFD9FF1200D9CFE6FFE1CFD9FF1D
:100AF00083E941E8036A080E035C09E20350EA6AED
:100B0000080FE96E000EEA22EF6A032AF4D7080EF6
:100B1000E66E000EE66E00EBE6FF01EBE6FFB0ECE2
:100B20001CF044E9080EE66E000EE66E22EC00F0C2
:100B300042E9E66AABDE41E900D042E9E7CFD9FFFE
:100B40001200D9CFE6FFE1CFD9FF82E941E800509A
:100B500025E00050090A1BE00E0A12E00F0A0AE025
:100B60000E0A01E01AD0010EE66E1DEC01F041E91B
:100B7000026E13D0E66A1DEC01F041E9026E0DD061
:100B8000010EE66EACEC01F041E9026E06D0E66AB9
:100B9000ACEC01F041E9026E00D023D0010EE66E0C
:100BA0001DEC01F041E9000103B113D0E66A1DEC30
:100BB00001F041E9000103B10CD0010EE66EACEC8E
:100BC00001F041E9000103B104D0E66AACEC01F0A8
:100BD00041E900010351010B02E0000E01D00D0EAE
:0E0BE000026E025000D042E9E7CFD9FF1200AA
:020BEE00000104
:100BF0000081009300850087016B3E6BC00E046F7F
:100C0000330E056FF10E066F320E026F12000001F7
:100C10000391F7EF05F0D9CFE6FFE1CFD9FF83E9E4
:100C200044E800EBE6FF01EBE6FF9FEC1FF042E932
:100C3000F3CF13F1F4CF14F10101060E131901E102
:100C4000145119E1D950030FE66EDACFE6FF00EB3D
:100C5000E6FF01EBE6FFB0EC1CF044E9030E035C99
:100C60000AE1C00E04140001046F05EB05F006EB69
:100C700006F0000E02D0010E00D045E9E7CFD9FF03
:100C80001200D9CFE6FFE1CFD9FF83E942E89C0EFD
:100C9000E66E2F0EE66E040E01010024136F000EA7
:100CA0000120146F13C1E6FF14C1E6FF55EC1FF0DD
:100CB00044E9000907E100EC19F0F350036EF45029
:100CC000046E06D023EC19F0F350036EF450046E5A
:100CD00003EBE6FF04EBE6FF46EC1BF042E943E9D9
:100CE000E7CFD9FF1200D9CFE6FFE1CFD9FF83E9E3
:100CF00042E800EBE6FF01EBE6FF9FEC1FF042E964
:100D0000F3CF13F1F4CF14F1010113510608000ED3
:100D1000145511E300EBE6FF01EBE6FF9FEC1FF03B
:100D200042E9F3CF15F1F4CF16F10101050E155D7F
:100D3000000E165902E2010E34D0040E0024E96EB2
:100D4000000E0120EA6EEF5041080CE1010E046E26
:100D5000050E0024E96E000E0120EA6EEF50D00F60
:100D6000036E0FD0040E0024E96E000E0120EA6E1F
:100D7000EF50D00F036E035002E1010E01D0000EC0
:100D8000046ED8900CE20350090809E304EBE6FF77
:100D900003EBE6FFBAEC19F042E9000E02D0010EB7
:100DA00000D043E9E7CFD9FF120000010391120000
:100DB000D9CFE6FFE1CFD9FF83E944E800EBE6FFB6
:100DC00001EBE6FF9FEC1FF042E9F350056EF45093
:100DD000066E060ED89006BE03D0055C000E0658BF
:100DE00025E3063404E205500708000E06541EE30E
:100DF000D950030FE66EDACFE6FF040E010100249E
:100E0000136F000E0120146F13C1E6FF14C1E6FF3B
:100E1000B0EC1CF044E9030409E104EB02F000012A
:100E2000025102E1320E026F000E02D0010E00D01C
:100E300045E9E7CFD9FF1200D9CFE6FFE1CFD9FFCF
:100E400084E941E8046A0250120A01E178D0010AFB
:100E500073E0020A69E0010A5FE01F0A55E0010A37
:100E60004BE0030A47E0010A42E0070A3DE0010ABD
:100E700032E0030A2BE0010A26E00E0A20E0010A14
:100E80001EE0020A19E0010A14E0070A0FE0010A55
:100E90000AE0030A05E0010A01E054D0A8DE54D0BC
:100EA0000001009151D0000100814ED0090E046E66
:100EB0004BD00001009548D00001008545D0A7DE49
:100EC000090E046E41D00A0E046E3ED0ADEC0BF05C
:100ED000080E046E39D000EBE6FF01EBE6FFD1DE31
:100EE00042E9080E046E30D0000100932DD00001BD
:100EF00000832AD05ADF28D000EBE6FF01EBE6FFA3
:100F00008ADE42E9046E20D000EBE6FF01EBE6FF4B
:100F1000EADE42E9046E18D000EBE6FF01EBE6FFE3
:100F2000E2DE42E9046E10D000EBE6FF01EBE6FFE3
:100F30003FDF42E9046E08D00E0E046E05D00F0E9E
:100F4000046E02D0010E046E045000D042E9E7CFD7
:100F5000D9FF1200D9CFE6FFE1CFD9FF82E90050D7
:100F60000F0A01E18ED0010A01E189D0060A01E1F0
:100F700085D0050A01E17AD0010A70E0070A66E02F
:100F80000C0A5CE0010A52E0030A48E0010A3EE074
:100F9000070A34E0090A30E0030A26E00B0A1CE0E5
:100FA000020A12E0010A08E0870EE66E4A0EE66EBB
:100FB00046EC1BF042E96DD0F40EE66E490EE66E8B
:100FC00046EC1BF042E965D0F60EE66E490EE66E81
:100FD00046EC1BF042E95DD0100EE66E4A0EE66E5E
:100FE00046EC1BF042E955D0F90EE66E490EE66E6E
:100FF00046EC1BF042E94DD008D94BD0340EE66EDA
:101000004A0EE66E46EC1BF042E943D03F0EE66E18
:101010004A0EE66E46EC1BF042E93BD04B0EE66E04
:101020004A0EE66E46EC1BF042E933D0530EE66EF4
:101030004A0EE66E46EC1BF042E92BD0590EE66EE6
:101040004A0EE66E46EC1BF042E923D0620EE66ED5
:101050004A0EE66E46EC1BF042E91BD06B0EE66EC4
:101060004A0EE66E46EC1BF042E913D0750EE66EB2
:101070004A0EE66E46EC1BF042E90BD00AD09ED831
:1010800008D0950EE66E4A0EE66E46EC1BF042E97D
:1010900000D09A0EE66E2F0EE66E00EC1BF042E9D1
:1010A00041E9E7CFD9FF1200D9CFE6FFE1CFD9FF61
:1010B00083E948E8036800EBE6FF01EBE6FF6EEC2E
:1010C0001DF042E900EBE9FF01EBEAFFEF5005E11B
:1010D0003E0E006E000E016E0BD000EBE6FF01EB42
:1010E000E6FF3E0EE66E000EE66E68EC1FF044E989
:1010F000020EE66EE66A970EE66E2F0EE66E00EBC7
:10110000E6FF01EBE6FFC0EC1EF046E9000909E04E
:1011100000EBE6FF01EBE6FFCEEC19F042E9046ECE
:1011200040D0040EE66EE66A00EBE6FF01EBE6FF58
:10113000D950060FE66EDACFE6FFADEC1FF046E9B8
:101140000A6A056A140EF36EF46AF350055C000E29
:10115000F4541EE2F76A0534FE0BF66EF7369B0E6A
:10116000F6264A0EF7220900F5CFE6FF0900F5CF73
:10117000E6FFD950060FE66EDACFE6FF55EC1FF01A
:1011800044E9000903E185EB03F002D0052ADAD730
:1011900000EBE6FF01EBE6FF03EBE6FF4DDE43E984
:1011A000046E04EBE6FFD6DE41E949E9E7CFD9FF5B
:1011B0001200000103911BDD8FEF14F0D9CFE6FF81
:1011C000E1CFD9FF81E942E8D950010FE66EDACFCD
:1011D000E6FF91EC1DF042E9150EE66E000EE66E9C
:1011E000020EE66ED950010FE66EDACFE6FFF4ECA0
:1011F0001CF045E9150EE66E000EE66E27EC1BF0BE
:1012000042E943E9E7CFD9FF1200D9CFE6FFE1CFAA
:10121000D9FF81E942E8D950010FE66EDACFE6FF47
:1012200091EC1DF042E9100EE66E4A0EE66E150EC8
:10123000E66E000EE66E89EC1FF044E9120E025CC9
:1012400010E1E00E011460080CE18A0EE66E2F0E2C
:10125000E66E150EE66E000EE66E28EC1FF044E911
:1012600031D0120E025C10E1E00E011440080CE1D6
:101270007D0EE66E2F0EE66E150EE66E000EE66E25
:1012800028EC1FF044E91ED0240E025C10E1E00EB1
:10129000011420080CE17D0EE66E2F0EE66E150E91
:1012A000E66E000EE66E28EC1FF044E90BD06A0EE5
:1012B000E66E2F0EE66E150EE66E000EE66E28EC5C
:1012C0001FF044E9150EE66E000EE66E27EC1BF0EB
:0A12D00042E943E9E7CFD9FF12001D
:0612DA00EB0ED76EDB0EE7
:1012E000D66EF2941200F2A4FED71200D9CFE6FF18
:1012F000E1CFD9FF82E90F0E00140A0A18E0040AB0
:1013000016E0070A12E0020A10E0060A0EE0020ADE
:101310000CE0090A08E0030A04E0020A02E0000EF9
:1013200008D0000E06D0000E04D0010E02D0000E30
:1013300000D041E9E7CFD9FF1200D9CFE6FFE1CFD6
:10134000D9FF82E943E800010391005007E0FE0E57
:10135000E66E4F0EE66E00EC1BF042E9AAEC15F0CB
:10136000026E025004E1070EF36EF46AACD0005036
:1013700007E0080EE66E500EE66E00EC1BF042E948
:10138000150EE66E4C0EE66E030EE66E080EE66E69
:10139000000EE66E09EC15F045E90001085104E184
:1013A000050EF36EF46A8FD0030E085D03E1550E4F
:1013B000095D04E0030EF36EF46A85D00A51036EF2
:1013C0000B51046E005007E0080EE66E500EE66EFC
:1013D00000EC1BF042E9270EE66E58EC27F041E9DD
:1013E0000001010E086F0B1D096F080EE66E000E5E
:1013F000E66EC9EC14F042E9026E025004E1070EF9
:10140000F36EF46A60D0150EE66E0D0EE66E010EF8
:10141000E66E080EE66E000EE66E09EC15F045E984
:101420000001085104E1050EF36EF46A4CD0080582
:1014300003E1CC0E095D04E0030EF36EF46A43D0C1
:10144000005007E0080EE66E500EE66E00EC1BF052
:1014500042E9080E045C03E0940E045C0DE1000117
:101460000051080B03E1030E015D05E1000103815A
:101470000001030E016F15D08F0E045C12E103EB27
:10148000E6FF34DF41E900090CE000010051080BE0
:1014900003E1040E015D05E1000103810001040E7A
:1014A000016F00010351010B02E0000E01D0050E97
:1014B0000101136F146B800B01E0146913C1F3FF7A
:1014C00014C1F4FF00D044E9E7CFD9FF1200D9CF0F
:1014D000E6FFE1CFD9FF82E943E800010391005024
:1014E00007E0FE0EE66E4F0EE66E00EC1BF042E9E2
:1014F00006EC16F0026E025002E1070E74D0020EE6
:10150000E66EE66AF60EE66E4F0EE66E080EE66EC4
:10151000000EE66E08EC1FF046E9E66A040EE66E81
:10152000000EE66E080EE66E000EE66E06EC24F087
:1015300045E9080EE66E000EE66EC6EC23F042E9C1
:10154000080EE66E000EE66EC9EC14F042E9320EAB
:10155000E66E4C0EE66E080EE66E080EE66E000EA7
:10156000E66E09EC15F045E90001085102E1050EAF
:101570003AD0050E085D02E2030E35D0095103E1B1
:10158000030E036E0ED0C00E091503E1020E036EAA
:1015900008D03F0E091503E0040E036E02D0050EBD
:1015A000036E0350EA6A080FE96E000EEA22EF505C
:1015B000C10802E0030E17D00328EA6A080FE96E9B
:1015C000000EEA22EF50046E04EBE6FF8FDE41E9E5
:1015D000000907E0000103810001050E016F000E04
:1015E00002D0030E00D044E9E7CFD9FF1200D9CFD3
:1015F000E6FFE1CFD9FF82E941E8005016E0005054
:10160000050A0CE0060A03E0070A01E00DD000EB32
:10161000E6FF93DE41E9F350026E06D000EBE6FFF1
:1016200056DF41E9026E00D011D0E66A86DE41E95C
:10163000000103B103D0E66A4ADF41E9000103512A
:10164000010B02E0000E01D00D0E026E000103A19D
:101650000ED043DE01012A690001076B005007E04C
:101660000A0EE66E500EE66E46EC1BF042E90250A2
:1016700000D042E9E7CFD9FF1200D9CFE6FFE1CF92
:10168000D9FF81E942E8030E0001015D16E1040E75
:10169000E66EE66AF80EE66E4F0EE66E080EE66E31
:1016A000000EE66E08EC1FF046E9080EE66E000E2E
:1016B000E66EAAEC23F042E91AD0020EE66EE66A64
:1016C000FC0EE66E4F0EE66E080EE66E000EE66E3F
:1016D00008EC1FF046E9E66A040EE66E000EE66EC0
:1016E000080EE66E000EE66E06EC24F045E9080EE4
:1016F000E66E000EE66EC6EC23F042E9F4DD080E5D
:10170000E66E000EE66EC9EC14F042E9016E01507F
:1017100003E10001072B1CD0026A150EE66E02C021
:10172000E6FF0B0EE66E080EE66E000EE66E09ECA6
:1017300015F045E90001085105E1025003E10001FF
:10174000072B06D0050E085D01E202D0022AE5D77C
:10175000C4DD43E9E7CFD9FF1200150EE66E000E97
:10176000E66E0D0EE66E080EE66E000EE66EF4EC0A
:101770001CF045E9150EE66E000EE66E27EC1BF038
:1017800042E9120000010751050802E2039112D05C
:10179000FF0E01012A5D04E1CE6ACF6A9E9008D057
:1017A0009EA002D02A2B9E903A0E2A5D01E202D022
:1017B0002A6B63DF1200CE6ACF6A9E9001012A6B0A
:1017C0000001076B1200D9CFE6FFE1CFD9FF83E913
:1017D00043E8046A080EE66E000EE66E00EBE6FFD4
:1017E00001EBE6FFB0EC1CF044E9030E0001015DE3
:1017F00008E1080EE66E000EE66EAAEC23F042E960
:101800000CD0E66A040EE66E000EE66E080EE66E7A
:10181000000EE66E06EC24F045E9080EE66E000EBA
:10182000E66EC6EC23F042E95EDD080EE66E000EC1
:10183000E66EC9EC14F042E9036E035002E10B0EB0
:1018400056D0150EE66E02C0E6FF0B0EE66E080ED1
:10185000E66E000EE66E09EC15F045E90001085150
:1018600004E1045040E1050E42D0050E085D02E29D
:10187000030E3DD0010E046E000100B31FD0080E10
:10188000E66E000EE66EF1EC23F042E9000108512D
:1018900002E1040E2CD0030E0001015D08E1080EE8
:1018A000E66E000EE66EDAEC23F042E907D0080E91
:1018B000E66E000EE66E45EC24F042E9150EE66E8B
:1018C000000EE66E08C0E6FF090EE66E000EE66E3C
:1018D000F4EC1CF045E9150EE66E000EE66E27EC02
:1018E0001BF042E9AED767DFF8DC080E00D044E910
:0618F000E7CFD9FF120052
:0A18F600D9CFE6FFE1CFD9FF83E967
:1019000041E88A8400EBE6FF01EBE6FF7AEC24F085
:1019100042E9036E8A94035000D042E9E7CFD9FF31
:101920001200D9CFE6FFE1CFD9FF81E942E8F2B456
:1019300041D080A2FCD7CF6ACE6A9E9080A203D00D
:101940009EB001D0FBD79EA002D0FF0E35D08AEC0E
:1019500027F0F350016EF450026E01EB13F102EB2D
:1019600014F10101156B166BD8901651000A08E6A8
:10197000F40E135D000E1459000E1559000E165981
:1019800018E301EB13F102EB14F1156B166B16352E
:10199000000E161909E6D880660E1355010E14556F
:1019A000000E1555000E165502E3010E01D0FF0E74
:1019B00003D0BDD7000E00D043E9E7CFD9FF120016
:1019C000D9CFE6FFE1CFD9FF84E949E881EB04F004
:1019D00082EB05F0A6DF076E070402E00750A0D0F7
:1019E000CF6ACE6A01EBE9FF02EBEAFFEF6A8A8277
:1019F000066A0050065C01E387D0080E0A6E0B6A87
:101A00000C6A0A500A06000970E00B9E0B468050D3
:101A1000020B01E0010E0C5C18E18AEC27F0F3CF19
:101A200013F1F4CF14F10101156B166BD890165118
:101A3000000A08E6F40E135D000E1459000E155945
:101A4000000E165901E360D0E2D78050020B01E08E
:101A5000010E0C6E8AEC27F0F350086EF450096EFC
:101A6000CF6ACE6A08EB13F109EB14F10101156B93
:101A7000166BD8901651000A08E6330E135D000E5F
:101A80001459000E1559000E165901E246D008EB04
:101A900013F109EB14F1156B166B1635000E1619C0
:101AA00009E6D880F40E1355000E1455000E155596
:101AB000000E165501E231D008EB13F109EB14F1D9
:101AC000156B166B1635000E161909E6D880900EA8
:101AD0001355000E1455000E1555000E165502E252
:101AE000010E01D0000E0B128CD7550E0B18E66EAE
:101AF000042A000E052204EBE9FF05EBEAFFE5529C
:101B0000E750EF6E062A75D701EBE9FF02EBEAFF1B
:101B100006EBEFFF8A92010E03D08A92FF0E00D0EF
:101B20004AE9E7CFD9FF1200D9CFE6FFE1CFD9FFCD
:101B300083E948E800010251056E0550AE0802E253
:101B4000AE0E056E770EE66E010EE66E0550E66E81
:101B5000E66A2DEC21F0FE0EE350FF08066EFF0E44
:101B600041E9E554076E080EE66E000EE66E00EBE6
:101B7000E6FF01EBE6FFB0EC1CF044E9080EE66E70
:101B8000000EE66E76EC1EF042E9080EE66E000EE0
:101B9000E66EE1EC1DF042E9080EE66E000EE66E20
:101BA000AADE42E9000A03E0FF0A01E002D00B0EC0
:101BB000CAD00A6A000E086E020E096E06EBE6FF36
:101BC00007EBE6FF9CEC27F042E9F294F2B463D015
:101BD0000B0EE66E08EBE6FF09EBE6FFF1DE43E9EC
:101BE000036EFF0E035C03E10C0E046EAAD00350DB
:101BF00001E151D00828E96E000E0920EA6EEFCF0E
:101C000013F14C0EF66E500EF76E0800F550010100
:101C1000135D10E1020E0824E96E000E0920EA6E41
:101C2000EFCF14F14D0EF66E500EF76E0800F55022
:101C3000145D01E02FD008EBE9FF09EBEAFFEFCFDD
:101C400013F1050E135D07E308EBE9FF09EBEAFF6B
:101C5000EF500B0801E21ED006EBE6FF07EBE6FFB4
:101C60009CEC27F042E908EBE9FF09EBEAFFEF28DB
:101C70000A2608EBE9FF09EBEAFFEF280826000E29
:101C80000922F40EF36EF46A0A50F35C000EF45865
:101C900001E201D09BD708EBE9FF09EBEAFFEF6A0D
:101CA000000E086E020E096E08EBE9FF09EBEAFF71
:101CB000EF5041E00D0EE66EE66A08EBE6FF09EB39
:101CC000E6FF080EE66E000EE66EDDEC1EF046E95D
:101CD000000100B313D0080EE66E000EE66E03ECB2
:101CE0001EF042E9000903E1040E046E2AD0080E3A
:101CF000E66E000EE66EDAEC23F042E9150EE66EB3
:101D0000000EE66E08C0E6FF090EE66E000EE66EF7
:101D1000F4EC1CF045E9150EE66E000EE66E27ECBD
:101D20001BF042E908EBE9FF09EBEAFFEF28082680
:101D3000000E0922B9D70A5002E1050E01D0080EA3
:101D4000046E045000D049E9E7CFD9FF1200D9CF83
:101D5000E6FFE1CFD9FF81E945E80001020E086FF7
:101D6000010E096F0A6B00010251036E0350AE08A9
:101D700002E2AE0E036E770EE66E010EE66E0350C3
:101D8000E66EE66A2DEC21F0FE0EE350FF08046ECD
:101D9000FF0E41E9E554056E080EE66E000EE66E94
:101DA00076EC1EF042E9080EE66E000EE66EE1ECFF
:101DB0001DF042E9080EE66E000EE66E9CDD42E97B
:101DC000000A03E0FF0A01E002D00B0E40D004EB52
:101DD000E6FF05EBE6FF9CEC27F042E9F294F2B453
:101DE00034D00B0EE66E080EE66E000EE66EE8DDF1
:101DF00043E9016EFF0E015C03E10C0E026E25D07B
:101E0000015003E1060E026E20D04C0EF66E500E0D
:101E1000F76E0800F5500001095D08E14D0EF66E01
:101E2000500EF76E0800F5500A5D01E00DD0070E68
:101E3000085D03E2030E026E08D000010381000179
:101E4000020E016F026A01D0CAD7025000D046E9E3
:061E5000E7CFD9FF1200EC
:0A1E5600D9CFE6FFE1CFD9FF83E901
:101E600041E88A8400EBE6FF01EBE6FFDBEC1FF0C4
:101E700042E9036E8A94035000D042E9E7CFD9FFCC
:101E80001200D9CFE6FFE1CFD9FF82E945E8026A27
:101E9000036A280EE66EE66AE66AE66A0050E66EB7
:101EA000E66AE66AE66A61EC21F0E552E5CF16F1F2
:101EB000E5CF15F1E5CF14F1E7CF13F1010113518F
:101EC000056E1451066ECE6AB4BC0FD0CE50960883
:101ED00004E2022A000E0322CE6A0250055C03507F
:101EE000065802E2000E03D0EFD7010E00D046E9FB
:101EF000E7CFD9FF1200D9CFE6FFE1CFD9FF85E9BF
:101F000041E800EBE6FFBDDF41E9000902E1000E18
:101F10000ED08A8201EBE6FF02EBE6FF03EBE6FF61
:101F20006CEC20F043E9056E8A92055000D042E93E
:101F3000E7CFD9FF1200D9CFE6FFE1CFD9FF83E980
:101F400048E800010251056E0550AE0802E2AE0EEF
:101F5000056E770EE66E010EE66E0550E66EE66AD9
:101F60002DEC21F0FE0EE350FF08066EFF0E41E956
:101F7000E554076E080EE66E000EE66E00EBE6FF17
:101F800001EBE6FFB0EC1CF044E9080EE66E000E33
:101F9000E66E2CEC1EF042E9080EE66E000EE66ED0
:101FA000E1EC1DF042E9080EE66E000EE66E53DF2E
:101FB00042E9FF0A08E0FF0A04E0010A01E005D057
:101FC00004D00C0ECED00B0ECCD00A6A000E086ED8
:101FD000020E096E06EBE6FF07EBE6FF9CEC27F02E
:101FE00042E9F294F2B465D005EBE6FF0C0EE66E22
:101FF00008EBE6FF09EBE6FF7EDF44E9036EFF0E28
:10200000035C03E10C0E046EAAD0035001E151D031
:102010000828E96E000E0920EA6EEFCF13F14E0E8C
:10202000F66E500EF76E0800F5500101135D10E1D9
:10203000020E0824E96E000E0920EA6EEFCF14F1BB
:102040004F0EF66E500EF76E0800F550145D01E06D
:102050002FD008EBE9FF09EBEAFFEFCF13F1050EF4
:10206000135D07E308EBE9FF09EBEAFFEF500B080C
:1020700001E21ED006EBE6FF07EBE6FF9CEC27F043
:1020800042E908EBE9FF09EBEAFFEF280A2608EB33
:10209000E9FF09EBEAFFEF280826000E0922F40EFB
:1020A000F36EF46A0A50F35C000EF45801E201D0BA
:1020B00099D708EBE9FF09EBEAFFEF6A000E086E1B
:1020C000020E096E08EBE9FF09EBEAFFEF5041E071
:1020D0000D0EE66EE66A08EBE6FF09EBE6FF080E7A
:1020E000E66E000EE66EDDEC1EF046E9000100B380
:1020F00013D0080EE66E000EE66E03EC1EF042E909
:10210000000903E1040E046E2AD0080EE66E000EEC
:10211000E66EDAEC23F042E9150EE66E000EE66E8E
:1021200008C0E6FF090EE66E000EE66EF4EC1CF049
:1021300045E9150EE66E000EE66E27EC1BF042E94F
:1021400008EBE9FF09EBEAFFEF280826000E092259
:10215000B9D70A5002E1050E01D0080E046E0450F2
:1021600000D049E9E7CFD9FF1200D9CFE6FFE1CF90
:10217000D9FF81E945E80001020E086F010E096FE1
:102180000A6B00010251036E0350AE0802E2AE0E6C
:10219000036E770EE66E010EE66E0350E66EE66A9B
:1021A0002DEC21F0FE0EE350FF08046EFF0E41E916
:1021B000E554056E080EE66E000EE66E2CEC1EF081
:1021C00042E9080EE66E000EE66EE1EC1DF042E913
:1021D000080EE66E000EE66E3EDE42E9FF0A05E0FE
:1021E000FF0A01E004D00C0E44D00B0E42D004EBE9
:1021F000E6FF05EBE6FF9CEC27F042E9F294F2B42F
:1022000036D003EBE6FF0C0EE66E080EE66E000E0F
:10221000E66E71DE44E9016EFF0E015C03E10C0E17
:10222000026E25D0015003E1060E026E20D04E0E44
:10223000F66E500EF76E0800F5500001095D08E1DA
:102240004F0EF66E500EF76E0800F5500A5D01E075
:102250000DD0070E085D03E2030E026E08D00001E8
:1022600003810001010E016F026A01D0C8D702503C
:0A22700000D046E9E7CFD9FF1200C5
:06227A006C500CE16896B7
:10228000040100513C0BE842E8420D0802E10ED87F
:1022900001D045D808D0040E6C5C03E168964FD895
:1022A00002D0000E02D0010E00D01200D9CFE6FFFE
:1022B000E1CFD9FF81E941E8040104BF046B0101CA
:1022C000126B0A6B0B6B106B116B2AEC16F0016A28
:1022D000010EF36EF46AF350015C000EF4541AE23E
:1022E00001010B5101E016D0F76A0134FE0BF66EC6
:1022F000F736700EF6264B0EF7220900F5CF13F1D4
:102300000800F5CF14F114C1FAFF010113511400B4
:10231000012ADED7CFD842E9E7CFD9FF1200020E5B
:1023200001010A5D0AE192D8040100BD03D0C80E84
:10233000006F02D0880E006F01D002D91200040E87
:1023400001011C5D0AE122C46EFF6E50000803E229
:10235000050E1C6F02D0030E1C6F01010A0512E16D
:1023600013D8020E0101125D04E10401840E046F12
:1023700008D0040104BD03D0C80E046F02D0880E3B
:10238000046F01D0DDD81200D9CFE6FFE1CFD9FF2D
:1023900081E942E80101080E105D000E11590EE2BC
:1023A0001051016E1151026E125103E1010E126FB4
:1023B00004D0120502E1020E126F03D0080E016E66
:1023C000026A0401049304910250041301EB05F422
:1023D00001500101105F0250115B280E0E6F040EB8
:1023E0000F6F01011DA318D00150021014E00CC1A1
:1023F000F6FF0DC1F7FF0800F5500EC1E9FF0FC150
:10240000EAFFEF6E01010E2B000E0F230C2B0D23A4
:102410000106025AE9D716D00150021013E00CC190
:10242000E9FF0DC1EAFFEF500EC1E9FF0FC1EAFF5E
:10243000EF6E01010E2B000E0F230C2B0D23010656
:10244000025AEAD743E9E7CFD9FF1200D9CFE6FF16
:10245000E1CFD9FF81E942E8030E04010015026EC5
:102460000151016E100EE96E010EEA6E0101EE508F
:102470000124106FED500220116F280E0C6F040E16
:102480000D6F0150021012E00CC1E9FF0DC1EAFF0F
:10249000EF500EC1E9FF0FC1EAFFEF6E0E2B000EE9
:1024A0000F230C2B0D230106025AEBD743E9E7CF8C
:1024B000D9FF12006D9801010B510CE10401080EC7
:1024C000016F200E026F040E036F840E006F040173
:1024D000046F35D0040120AF22D001011051040156
:1024E000265D010111510401275904E226C410F1AF
:1024F00027C411F149DF0101010E0A6F0401080E22
:10250000016F200E026F040E036F800E006F040136
:10251000280E066F040E076FC80E046F10D001015D
:10252000020E0A6F0401056BC80E046F0401080E49
:10253000016F280E026F040E036FC80E006F1200A9
:10254000D9CFE6FFE1CFD9FF81E941E8020E0101D1
:102550000A5D38E16D50100B35E0040101510101B5
:10256000136F146B080E131901E114512BE10401D0
:1025700000513C0BE842E8420D0824E10051800B79
:1025800021E1200E026F040E036F016A080EF36E44
:10259000F46AF350015C000EF45413E20150EA6A4D
:1025A000280FE96E040EEA22EF50E66E0150EA6A47
:1025B000200FE96E040EEA22E552E750EF6E012A81
:1025C000E5D70DD001010A6B0401080E016F200E42
:1025D000026F040E036F8C0E006F0401046B42E95E
:0625E000E7CFD9FF120055
:0A25E600040120511F0B010801E061
:1025F0005BD02051600BE842E842E842E842E84202
:10260000010801E051D0245103E0240501E04CD041
:102610002151230A48E0010A40E0030A30E0010AA0
:1026200025E0240A22E0070A1FE0010A1CE0030A51
:1026300011E0010A01E038D00101030E0B6F010126
:10264000F10E0C6F000E0D6F01011D930101080EBC
:10265000106F2AD00101030E0B6F0101F10E0E6FF6
:10266000000E0F6F21D020D01FD01ED00101030E0D
:102670000B6F0101E90E0E6F000E0F6F15D00101F7
:10268000030E0B6F0101E90E0C6F000E0D6F0101BF
:102690001D930101070E106F07D00101030E0B6F90
:1026A00022C4F0F001D000D012000001E96BC20E8C
:1026B000EA6F010EEB6FEC6BED6BEE6B080EEF6FDC
:1026C000E26BE16B1A0E726E1E0E736E0401000E49
:1026D000166F050E176F400E146F0401196F080E68
:1026E0001A6F050E1B6F880E186F0401480E1E6FBF
:1026F000050E1F6F400E1C6F1200D9CFE6FFE1CF11
:10270000D9FF84E90001E16B040118BF24D0005017
:10271000195D02E21951006E0001E16B0050E15DAC
:1027200013E2E151EA6A080FE96E050EEA22EF5062
:10273000E66EE1510124E96E000E0220EA6EE552D8
:10274000E750EF6EE12BEAD70401400E196F18171E
:10275000187D880E18130001E15100D041E9E7CF40
:10276000D9FF1200D9CFE6FFE1CFD9FF83E941E8D5
:102770000001E25101E022D0036A032AFF0EF36E4A
:10278000F46AF350031801E1F45001E109D000EBC1
:10279000E9FF01EBEAFF002A000E0122EF50EDE114
:1027A0000350005E000E015A00EBE3F001EBE4F091
:1027B00003040001E76FE86B010EE26F42E9E7CF27
:1027C000D9FF1200D9CFE6FFE1CFD9FF83E941E875
:1027D0000001E25101E023D0036A032AFF0EF36EE9
:1027E000F46AF350031801E1F45001E10AD000EB60
:1027F000F6FF01EBF7FF002A000E01220800F5505A
:10280000ECE10350005E000E015A00EBE3F001EB37
:10281000E4F003040001E76F010EE86FE26F42E9A4
:10282000E7CFD9FF1200D9CFE6FFE1CFD9FF81E989
:1028300041E804011CBF6FD0030E0001E25D01E11D
:10284000E26BE25101E167D0020EE25D06E10401B4
:102850001D6B0001030EE26F58D0E20556E1E7510F
:102860000101136F146B13514008000E145503E25D
:10287000400E016E03D00001E751016E01EB1DF423
:1028800001500001E75DE76F480EE56F050EE66F4A
:10289000E80515E1015012E0E3C0F6FFE4C0F7FFE0
:1028A0000800F550E5C0E9FFE6C0EAFFEF6EE52B52
:1028B000000EE623E32BE4230106ECD713D00150EE
:1028C00011E0E3C0E9FFE4C0EAFFEF50E5C0E9FF33
:1028D000E6C0EAFFEF6EE52B000EE623E32BE423D0
:1028E0000106EDD7E75111E104011D510101136FFC
:1028F000146B400E131901E1145104E10001020EA2
:10290000E26F03D00001030EE26F400E04011C17BA
:0E2910001C7D880E1C1342E9E7CFD9FF120090
:02291E00080EA1
:10292000B86E800EE66E040EE66E3C0EE66E5CEC53
:1029300026F043E91200D9CFE6FFE1CFD9FF81E9C4
:1029400041E8ABA206D0AE50016EAE50016EAB981E
:10295000AB8842E9E7CFD9FF1200D9CFE6FFE1CF3C
:10296000D9FF82E9FE0ED76E880ED66EF2949EBA1B
:1029700005D0F2A402D0000E08D0F9D70050AE5C0A
:1029800002E0000E01D0010E00D041E9E7CFD9FFEF
:102990001200D9CFE6FFE1CFD9FF83E944E880EB0D
:1029A00004F081EB05F0010E066EC5DF8A8400EBB2
:1029B000E9FF01EBEAFFEF04036E033423E2ACA26C
:1029C000FED7042A000E052204EBE9FF05EBEAFF1F
:1029D000EF50AD6E04EBE9FF05EBEAFFEFCFE6FF4A
:1029E000BCDF41E9000902E1066A0CD0033402E2CF
:1029F0000350000805E2540EE66ED2EC27F041E9E0
:102A00000306DBD78A94065000D045E9E7CFD9FF0B
:102A10001200D9CFE6FFE1CFD9FF86E945E8066A83
:102A200083EB09F084EB0AF0F2940150AE0802E265
:102A3000AE0E016E01500101136F146B770E14037B
:102A4000F3CF14F113511427770E1303F3CF13F1BF
:102A5000F4501427FF0ED8801357145714C113F1E4
:102A6000146B13C1D7FF0150136F146B770E14034F
:102A7000F3CF14F113511427770E1303F3CF13F18F
:102A8000F4501427FF0ED880135714571351D66EE5
:102A9000040EE66EE66A770EE66E010EE66E0050F4
:102AA000E66EE66A2DEC21F0F1EC20F0E552E5CF80
:102AB00014F1E7CF13F10101FF0ED880135714571B
:102AC00014C113F1146B1351076E040EE66EE66A1F
:102AD000770EE66E010EE66E0050E66EE66A2DECAD
:102AE00021F0F1EC20F0E552E5CF14F1E7CF13F13E
:102AF0000101FF0ED880135714571351086E03EBD2
:102B0000E9FF04EBEAFFEF6A066A0250065C17E28F
:102B10009EBA03D0F2B413D0FBD7ABB210D0092ABF
:102B2000000E0A2209EBE9FF0AEBEAFFAECFEFFF46
:102B30008A8207EBD7FF08EBD6FF062AE6D703EB1E
:102B4000E9FF04EBEAFF06EBEFFF8A9246E9E7CFE5
:102B5000D9FF1200F0DE8A84AB9EAC9A8B9C8A8AE5
:102B6000F00EE66E58EC27F041E98B8C8A9AF00E55
:102B7000E66E58EC27F041E98B8C8A9AF00EE66EEF
:102B800058EC27F041E98B9C8A8AF00EE66E58ECEF
:102B900027F041E98B9C8A8AF00EE66E58EC27F00C
:102BA00041E98B8C8A9AF00EE66E58EC27F041E9E9
:102BB0008B8C8A9AF00EE66E58EC27F041E98B9CDC
:102BC0008A8AF00EE66E58EC27F041E98B9C8A8ADF
:102BD000F00EE66E58EC27F041E98B8C8A9AF00EE5
:102BE000E66E58EC27F041E9AB8EAC8A8A9482BE3F
:102BF00002D0000E0AD0000100A905D0E668ADDEC3
:102C000041E903D002D0010E00D0120094DE8A8484
:102C1000AB9EAC9A8B9C8A8A1E0EE66E58EC27F00F
:102C200041E98B8C8A9A1E0EE66E58EC27F041E93A
:102C3000AB8EAC8A8A9482BE02D0000E0AD000010C
:102C400000A905D0E66889DE41E903D002D0010E73
:042C500000D012009E
:0C2C540004012051600BE842E842E84215
:102C6000E842E842000901E054D02151070A50E04F
:102C70000B0A4EE0070A3FE0010A2CE00B0A28E0AD
:102C8000020A26E0030A22E0080A12E0010A0EE026
:102C90000F0A0AE0030A01E03BD00101010E0B6FAD
:102CA0000101040E1C6F35D035D833D08FD831D008
:102CB0000101010E0B6F01011E0E0C6F010E0D6F55
:102CC00001011D930101010E106F23D0A3D821D063
:102CD000F4D81FD00101010E0B6F04012451010132
:102CE0000D6B1F0F0C6F010E0D2301011D930101D0
:102CF000010E106F0ED00101010E0B6F0401245163
:102D0000EA6A1F0FE96E010EEA2222C4EFFF01D02A
:102D100000D01200800E0401205D57E12351030A08
:102D200034E0010A10E0030A01E04DD00101010E78
:102D30000B6F0101C30E0C6F4A0E0D6F120E0101D5
:102D4000106F116B40D00101010E0B6F0401225175
:102D5000F66EF76AD890F636F736640EF6264B0E06
:102D6000F7220900F5CF0CF10A00F5CF0DF1020EA4
:102D70000101F76A0C25F66E0D51F7220900F5CF17
:102D800010F10A00F5CF11F11ED00101010E0B6FF9
:102D900004012251F66EF76AD890F636F736680EBF
:102DA000F6264B0EF7220900F5CF0CF10A00F5CFFD
:102DB0000DF10CC1F6FF0DC1F7FF0800F550010140
:102DC000106F116B00D001011D8312000101010E73
:102DD0000B6F0F0EE66E710EE66E0F0EE66E98EC40
:102DE00023F043E9010EE66E1F0EE66E010EE66E5D
:102DF00098EC23F043E922C41EF10401225104E1BE
:102E00000101050E1C6F05D00101060E1C6F55EC6B
:102E100013F012000401286B296B040120511F0BD1
:102E2000020A14E0030A0EE0010A01E038D00101B1
:102E3000010E0B6F0401288101011DA102D00401C4
:102E400028832DD00101010E0B6F29D00101010E45
:102E50000B6F040124510F0B080DF3500101146B8B
:102E6000000F136F040E142304012451800B01E0A2
:102E7000010E040DF3500101132501010E6F000E28
:102E80000101142101010F6F0EC1E9FF0FC1EAFF1B
:102E9000EF50040B03E00401010E286F00D0010184
:102EA0000B050AE10101280E0C6F040E0D6F0101E4
:102EB0001D930101020E106F12000401220510E1A2
:102EC00020511F0B00090CE10101010E0B6F030ED5
:102ED0000401215D03E101011D8102D001011D9169
:102EE0000401225140E120511F0B02083CE1245112
:102EF0000F0B000938E00101010E0B6F0401245192
:102F00000F0B080DF3500101146B000F136F040E2B
:102F1000142304012451800B01E0010E040DF35031
:102F20000101132501010E6F000E010114210101A1
:102F30000F6F030E0401215D07E1840E0EC1E9FF4E
:102F40000FC1EAFFEF6E0FD024AF07D0400E0EC1C5
:102F5000E9FF0FC1EAFFEF6E06D0880E0EC1E9FF50
:082F60000FC1EAFFEF6E120041
:082F680020002C20756E73752A
:102F700070706F727465642063686970002C2050F3
:102F8000494331384632353530002C2050494331E1
:102F9000384632343535004154003E004E0041542D
:102FA000403200415452560041545354004154544D
:102FB0005000415453500041545348004154504331
:102FC00000415448310041544830004154445000BD
:102FD0004154424400415440310041545A0041544C
:102FE00057530041544C310041544C300041544936
:102FF00000415445310041544530004154440042A1
:103000005553494E49543A204F4B00425553494E6F
:1030100049543A202E2E2E4F4B00413900413800A2
:103020004137004136004135004134004133004111
:1030300032004131003900380037003600350034A5
:103040000033003200310030004155544F2C2049EC
:10305000534F2031353736352D34202843414E200B
:1030600032392F32353029004155544F2C204953E5
:103070004F2031353736352D34202843414E20310D
:10308000312F32353029004155544F2C2049534FB0
:103090002031353736352D34202843414E20323902
:1030A0002F35303029004155544F2C2049534F20A3
:1030B00031353736352D34202843414E2031312FDC
:1030C00035303029004155544F2C2049534F203181
:1030D000343233302D3420284B575020464153543E
:1030E00029004155544F2C2049534F20313432335D
:1030F000302D3420284B575020354241554429006B
:103100004155544F2C2049534F20393134312D3201
:10311000004155544F2C20534145204A3138353019
:1031200020565057004155544F2C20534145204ABA
:10313000313835302050574D0049534F2031353705
:1031400036352D34202843414E2032392F32353048
:10315000290049534F2031353736352D3420284347
:10316000414E2031312F323530290049534F203123
:10317000353736352D34202843414E2032392F350E
:103180003030290049534F2031353736352D342022
:103190002843414E2031312F353030290049534FDB
:1031A0002031343233302D3420284B5750204641C3
:1031B0005354290049534F2031343233302D3420B9
:1031C000284B5750203542415544290049534F2040
:1031D000393134312D3200534145204A31383530B0
:1031E0002056505700534145204A31383530205041
:0F31F000574D004155544F000D000D0A000A00C5
:10320000D9CFE6FFE1CFD9FF81E941E800010151C3
:10321000016E00A702D00A0E0126EA6A0134FE0BF5
:10322000E96EEA368F0EE926000EEA22EECF13F1A0
:10323000EFCF14F113C1F3FF14C1F4FF00D042E942
:10324000E7CFD9FF1200D9CFE6FFE1CFD9FF81E95F
:1032500041E800010151016E00A702D00A0E0126CB
:10326000EA6A0134FE0BE96EEA36670EE926000EC3
:10327000EA22EECF13F1EFCF14F113C1F3FF14C123
:10328000F4FF00D042E9E7CFD9FF1200D9CFE6FF23
:10329000E1CFD9FF81E941E8060E016E000101513D
:1032A000060A20E0010A1EE00F0A1CE0010A1AE0EB
:1032B0000A0A11E0070A0FE0010A0DE0070A07E019
:1032C000030A01E016D0B5EC10F0016E12D0A7ECA5
:1032D0000EF0016E0ED001C0E6FFF7EC0AF041E9F6
:1032E000016E07D001C0E6FFA1EC05F041E9016ED7
:1032F00000D0015006E00001015105E00051080B2B
:1033000002E1015033D0B5EC10F0016E015001E143
:1033100013D0A7EC0EF0016E015001E10DD0E66A6A
:10332000F7EC0AF041E9016E015001E105D0E66ACF
:10333000A1EC05F041E9016E015016E1030E000118
:10334000015D08E10B0EE66E300EE66E46EC1BF0FA
:1033500042E90AD0030E015D07E1FF0EE66E2F0E73
:10336000E66E46EC1BF042E9015000D042E9E7CF9F
:10337000D9FF1200D9CFE6FFE1CFD9FF83E9015091
:1033800002E1010E01D0005000010097E8B0008773
:1033900001EB01F041E9E7CFD9FF1200D9CFE6FFF9
:1033A000E1CFD9FF83E941E800EBE6FF01EBE6FF5F
:1033B00083EC1CF042E9000902E1010E45D0000156
:1033C00003B107D063DF036E000103B102D00350E5
:1033D0003BD000010151060A2CE0010A2AE00F0A45
:1033E00028E0010A26E00A0A1BE0070A19E0010AA0
:1033F00017E0070A0CE0030A01E024D000EBE6FF27
:1034000001EBE6FF9BEC0FF042E9036E1BD000EBF3
:10341000E6FF01EBE6FF94EC0DF042E9036E12D0FB
:1034200000EBE6FF01EBE6FFE3EC0BF042E9036E95
:1034300009D000EBE6FF01EBE6FF74EC05F042E992
:10344000036E00D0035000D042E9E7CFD9FF12004D
:10345000000103A10BD000010151030A05E0070A96
:0E34600003E0010A01E002D0C2EC0BF0120002
:02346E0001015A
:103470002651271104E1200E266F4E0E276F2607D6
:10348000000E275B6DA205D02651271101E18A703D
:1034900006D001011C5102E18A9001D08A801200FD
:1034A000D9CFE6FFE1CFD9FF81E945E8E0DF060E9D
:1034B00001011C5D03E36D50020B01E06BD0B80EFF
:1034C000E66E000EE66E9FEC1FF042E9F350016ECF
:1034D000F450026EB80E0124036E000E0220046E3A
:1034E000010101502908136F000E0254146F13C11B
:1034F000E6FF03EBE6FF04EBE6FF7DEC13F043E9A8
:10350000056E055047E005500126000E0222290EE7
:10351000015C000E025803E30001B86B3BD0B80E0B
:103520000124E96E000E0220EA6EEF6A000100A19C
:1035300006D003EBE6FF04EBE6FF3BD842E90D0EB5
:10354000E66EB80EE66E000EE66E41EC1FF043E943
:10355000F350036EF450046E035004101BE000019E
:103560000051010B09E00051040B06E0FD0EE66E70
:10357000310EE66E45D842E903EBE9FF04EBEAFFC2
:10358000EF6AB80EE66E000EE66E54EC08F042E903
:103590000001B86B46E9E7CFD9FF12000001B86B14
:1035A0001200D4EC22F06FBE02D0F3EC22F013EF45
:1035B00014F0D9CFE6FFE1CFD9FF83E942E8036AEF
:1035C000046A0001E25110E0ECDF032A000E04223D
:1035D00003EB13F104EB14F101011351E808030E9E
:1035E000145501E209D0EDD700EBE6FF01EBE6FF51
:1035F000B2EC13F042E9D5DF43E9E7CFD9FF12007F
:10360000D9CFE6FFE1CFD9FF83E942E8036A046A34
:103610000001E25110E0C5DF032A000E042203EB93
:1036200013F104EB14F101011351E808030E1455D2
:1036300001E209D0EDD700EBE6FF01EBE6FFE2EC9B
:1036400013F042E9AEDF43E9E7CFD9FF1200D9CF4B
:10365000E6FFE1CFD9FF83E900EBE6FF01EBE6FFF0
:10366000A8DF42E9000100A507D0FA0EE66E310E90
:10367000E66EC6DF42E906D0F80EE66E310EE66E63
:10368000BFDF42E941E9E7CFD9FF1200D9CFE6FF1A
:10369000E1CFD9FF83E900EBE6FF01EBE6FF150E72
:1036A000E66E000EE66E89EC1FF044E9150EE66E3C
:1036B000000EE66ECCDF42E941E9E7CFD9FF120008
:1036C000D9CFE6FFE1CFD9FF8BE942E800EBE6FF77
:1036D00001EBE6FF02EBE6FF12EC28F043E907EB13
:1036E00013F1800E01011317146B156B1351141194
:1036F000151102E107EC28F0800EE66EAEEC27F023
:1037000041E90B6A0C6AC0EC27F080080EE00B2A36
:103710000B50F9E1800EE66EAEEC27F041E90C2A81
:10372000050E0C5CF0E1FF0E82D0C4D8100EBAD8A2
:1037300003E00101CBD8FEE1070EDDD8238F23C1C2
:10374000E6FF0F0EBED804EBE6FF05EBE6FF06EB47
:10375000E6FF71D843E9AED80C0EA4D803E001010E
:10376000B5D8FEE1070EC7D8E66E0D0EC9D8080E13
:1037700099D803E00101AAD8FEE10F0EBCD89AD86F
:10378000010E90D807E00101D89013371437153790
:10379000E806FAE1300E010113150101231323C1DC
:1037A000E6FF0C0EADD8600E01011617176B186BF3
:1037B000161F171F181F07EB19F108EB1AF109EB79
:1037C0001BF1040E19171A6B1B6B16511911136F8D
:1037D00017511A11146F18511B11156F13C123F1D2
:1037E00013C1E6FF600E8CD8050E5CD807E001011E
:1037F000D890133714371537E806FAE10101131F83
:10380000141F151F600E1317146B156B13C123F1D2
:1038100013C1E6FF700E55D8031C0101236FE66A41
:103820002C0E4FD823C1E6FF2B0E4BD8000E43E9D8
:10383000E7CFD9FF1200D9CFE6FFE1CFD9FF84E966
:1038400000EB24F10101241D256FE66E2A0E39D804
:103850004BD8080E27D803E0010138D8FEE113C188
:1038600024F10101241D3F0B0101136FC00E34D858
:10387000290E27D839D8100E15D803E0010126D813
:10388000FEE113C124F1470E01012417241D060B8C
:103890000101136F410E20D8280E13D841E9E7CF5C
:1038A000D9FF12001F0B16C113F117C114F118C173
:1038B00015F1120007EB16F108EB17F109EB18F1FF
:1038C0001200E66E3AEC27F042E91200D890153368
:1038D00014331333E80612000101241501011311FA
:1038E0000101256FE66E120000EB16F101EB17F1F6
:1038F00002EB18F11200010113150101236F1200F0
:06390000E0DF5AEF1CF0AD
:0A390600FE0EE3CFE9FFFF0EE3CF52
:10391000EAFFF36AEE5006E018D8FCE009D806E1A9
:10392000F32AF8D7F3B002D0F3501200E86A12007D
:10393000F452C60F0A0F06E2F450B90F060F02E266
:10394000D8941200F450D8841200F46E200806E0D7
:10395000F450090803E0F450D8941200D8841200FF
:10396000D9CFE6FFDACFE6FFFC0EE3CFE9FFFD0E8D
:10397000E3CFEAFFFC0EE3CFD9FFFD0EE3CFDAFF82
:10398000F36ADE5007E0E1DFFCE0D2DF1FE1F32A5B
:10399000EE6EF7D7EF6AF3B019D0F342FC0EE3CF27
:1039A000E9FFFD0EE3CFEAFFFA0EE3CFD9FFFB0EEE
:1039B000E3CFDAFFF3CFDEFFEF5206E00FD8E83AAD
:1039C000DF6E0CD8DE12F8D7F35001D0E86AE5526A
:1039D000E7CFDAFFE552E7CFD9FF1200EE50C00F74
:1039E000D8A0070F090F1200D9CFE6FFDACFE6FF04
:1039F000FC0EE3CFE9FFFD0EE3CFEAFFFB0EE3CFC2
:103A0000F3FFF90EE3CFD9FFFA0EE3CFDAFFF3525B
:103A10000FE0EF50F00BE83A12D8DE6EEE500F0BCD
:103A20000ED8DE6E200EDE6EF32EF3D7DD52DF6A87
:103A3000E552E7CFDAFFE552E7CFD9FF1200360FA4
:103A4000D8B2070FFA0F1200D9CFE6FFDACFE6FFA0
:103A5000F80EE3CFD9FFF90EE3CFDAFFF70EE3CF8D
:103A6000E8FFE86610D0FB0EE3CFE8FF33D8FA0E8C
:103A7000E3CFE8FF26D8DF6AE552E7CFDAFFE55269
:103A8000E7CFD9FF030CFD0EE3CFE8FF1AD8200ED5
:103A9000DE6EFC0EE3CFE8FF14D8200EDE6EFB0EC8
:103AA000E3CFE8FF0ED8200EDE6EFA0EE3CFE8FF7C
:103AB00008D8DF6AE552E7CFDAFFE552E7CFD9FF52
:103AC0000B0CE8CFE6FFF00BE83AB9DFDE6EE5520B
:103AD000E7CFE8FF0F0BB3DFDE6E1200D9CFE6FFB2
:103AE000DACFE6FFFC0EE3CFE9FFFD0EE3CFEAFFFE
:103AF000FC0EE3CFD9FFFD0EE3CFDAFFEE5009E075
:103B000024DFFCE0850F1A0FD8A0200F410FDE6ED6
:103B1000F5D7DE6EE552E7CFDAFFE552E7CFD9FF02
:103B20001200FE0EE3CFE9FFFF0EE3CFEAFF3F0EE8
:103B3000F86EFF0EF76EFE0EF66E0900F5CFEEFF83
:083B40000900F5CFEEFF1200B1
:083B4800D9CFE6FFE1CFD9FF60
:103B500083E946E880EB03F081EB04F000EBE9FF3A
:103B600001EBEAFFEF50056E0668055005060009F7
:103B700022E0080E076E032A000E042203EBE9FF81
:103B800004EBEAFFEF50086E07500706000912E049
:103B900008500618800B07E00E0E061A0650E8249F
:103BA0000109066E03D00650E824066E0850E8248A
:103BB000086EEAD7DAD7061C00D047E9E7CFD9FF6D
:103BC0001200D9CFE6FFE1CFD9FF83E941E800EB4E
:103BD000E6FF01EBE6FFB8DF42E9036E00EBE9FF29
:103BE00001EBEAFFEF2A00EBE9FF01EBEAFFEF5000
:103BF0000024E96E000E0120EA6E03EBEFFF42E9BC
:103C0000E7CFD9FF1200D9CFE6FFE1CFD9FF83E993
:103C100042E800EBE9FF01EBEAFFEF500024E96E18
:103C2000000E0120EA6EEF50036E00EBE9FF01EB9E
:103C3000EAFFEF0600EBE6FF01EBE6FF85DF42E976
:103C4000046E0450035C02E0000E01D0010E00D0AF
:103C500043E9E7CFD9FF1200D9CFE6FFE1CFD9FF83
:103C600083E941E800EBE9FF01EBEAFFEF50036E67
:103C70000350E66EE66A01010028136F000E012072
:103C8000146F13C1E6FF14C1E6FF040E0024156F84
:103C9000000E0120166F15C1E6FF16C1E6FFDDEC30
:103CA0001EF046E90028E96E000E0120EA6E610E62
:103CB000EF6E020E0024E96E000E0120EA6E6A0E1D
:103CC000EF6E030E0024E96E000E0120EA6EF10E85
:103CD000EF6E0101030E136F00EBE9FF01EBEAFF4A
:103CE0001351EF2642E9E7CFD9FF1200D9CFE6FF03
:103CF000E1CFD9FF83E941E800EBE9FF01EBEAFFFF
:103D0000EF50036E0350E66EE66A01010028136F60
:103D1000000E0120146F13C1E6FF14C1E6FF040E6C
:103D20000024156F000E0120166F15C1E6FF16C1A5
:103D3000E6FFDDEC1EF046E90028E96E000E0120EA
:103D4000EA6E680EEF6E020E0024E96E000E01208E
:103D5000EA6E6A0EEF6E030E0024E96E000E01207B
:103D6000EA6EF10EEF6E0101030E136F00EBE9FF37
:103D700001EBEAFF1351EF2642E9E7CFD9FF12002A
:103D8000FC0EE3CFF6FFFD0EE3CFF7FFFE0EE3CF11
:103D9000E9FFFF0EE3CFEAFFFA0EE35003E1FB0E6B
:103DA000E35009E0FA0EE30602E2FB0EE306090027
:103DB000F550EE5CF1E0F36E1200D9CFE6FFDACFFA
:103DC000E6FFFA0EE3CFD9FFFB0EE3CFDAFFFC0EDE
:103DD000E3CFE9FFFD0EE3CFEAFFE9CFF3FFEACF40
:103DE000F4FFF80EE35003E1F90EE35008E0F80E9B
:103DF000E30602E2F90EE306DECFEEFFF2D7FF0E96
:103E0000E3CFDAFFE552FF0EE3CFD9FFE552120010
:103E1000FC0EE3CFF6FFFD0EE3CFF7FFFE0EE3CF80
:103E2000E9FFFF0EE3CFEAFFE9CFF3FFEACFF4FFAC
:103E3000FA0EE35003E1FB0EE35009E0FA0EE3064D
:103E400002E2FB0EE3060900F5CFEEFFF1D7120008
:103E5000FC0EE3CFF6FFFD0EE3CFF7FFFE0EE3CF40
:103E6000E9FFFF0EE3CFEAFFE9CFF3FFEACFF4FF6C
:103E7000EE66FED7ED520900F5CFEFFFEE66FBD7F9
:103E80001200FE0EE3CFE9FFFF0EE3CFEAFFFD0EC7
:103E9000E350EF5C05E0EE66FAD7F36AF46A04D00B
:103EA000E9CFF3FFEACFF4FF1200FC0EE3CFF6FFF9
:103EB000FD0EE3CFF7FFFE0EE3CFE9FFFF0EE3CFEA
:103EC000EAFF0900F550EF5C02E1EE66FAD7120056
:103ED000D9CFE6FFDACFE6FFFA0EE3CFD9FFFB0E2C
:103EE000E3CFDAFFFC0EE3CFE9FFFD0EE3CFEAFFFD
:103EF000E9CFF3FFEACFF4FFDECFEFFFEE66FCD7AA
:103F0000FF0EE3CFDAFFE552FF0EE3CFD9FFE55214
:103F10001200FC0EE3CFF6FFFD0EE3CFF7FFFE0E1F
:103F2000E3CFE9FFFF0EE3CFEAFFE9CFF3FFEACFEC
:103F3000F4FF0900F5CFEFFFEE66FBD71200FE0E8F
:103F4000E3CFE9FFFF0EE3CFEAFFF36AF46AEE5234
:103F500003E0F34AF42AFBD71200D9CFE6FFDACF09
:103F6000E6FFFA0EE3CFD9FFFB0EE3CFDAFFFC0E3C
:103F7000E3CFE9FFFD0EE3CFEAFFE9CFF3FFEACF9E
:103F8000F4FFF80EE35003E1F90EE3500BE0F80EF6
:103F9000E30602E2F90EE306DECFEFFFEE66F1D7AD
:103FA000DD52EFD7FF0EE3CFDAFFE552FF0EE3CF8E
:063FB000D9FFE5521200EA
:0A3FB600E9CFE6FFEACFE6FFFC0EBC
:103FC000E3CFE9FFFD0EE3CFEAFF43E8D9CFE6FFF9
:103FD000DACFE6FFE1CFD9FFE2CFDAFF87E9EE5093
:103FE000026E025217E016E6B9D8000911E040D877
:103FF000EE50046E1DD800090BE0022EF9D70A0E10
:1040000040D84BD8000902E601E004D0E86A03D0AA
:10401000FF0E01D0010EE552E5CFDAFFE7CFD9FF61
:1040200043E9E552E7CFEAFFE552E7CFE9FF1200A7
:10403000080E036E04AE0AD000008A888A96080E25
:1040400020D88A988A860E0E1CD809D08A888A962B
:10405000100E17D88A988A86060E13D800D0B4BCE2
:10406000000C034E03D0044600D0E4D700D0010C6E
:104070008A888A96200E05D88A988A860F0E01D8DB
:104080001200E84E05D000D000D000D000D0F9D703
:10409000000000D000D000D01200CC6A046A080EE4
:1040A000036E0446B4BC05D0CC505108D8A012D041
:1040B000F9D7CC6AB4AC05D0CC503908D8A00BD015
:1040C000F9D7CC502408D8A002D0010E0412032E38
:1040D000E8D7010C000CFF0CE9CFE6FFEACFE6FFC2
:1040E000FC0EE3CFE9FFFD0EE3CFEAFFFB0EE3CFCB
:1040F000E8FF44E8D9CFE6FFDACFE6FFE1CFD9FF0A
:10410000E2CFDAFF88E9026EEE6A42D8000916E0D3
:1041100017E6056AC2DF000906E012E604EBEEFFCF
:10412000052A022EF7D70A0EACDFF10E81DF05500B
:10413000E82AE86C05EBEBFF010E03D0000E01D07E
:10414000FF0EE552E5CFDAFFE7CFD9FF44E9E552AC
:10415000E7CFEAFFE552E7CFE9FF1200DB0ED76EAB
:10416000600ED66EF294B4AC03D0F2B410D0FBD78C
:104170002D0ECC6E9E92B4BCF8D79EA2FCD7B10E89
:10418000CC6E9E92B4BC02D09EA2FCD7010C000C57
:10419000046AB4BC03D0F2B415D0FBD7CC6A9E92AB
:1041A000B4AC03D09EB210D0FBD75A0ECC5CF1E376
:1041B000CC5069080480EDE3B4BCEBD78A0ECC5C2C
:0A41C000FBE3010C04A0000CFF0C4F
:0641CA0043E8D9CFE6FF37
:1041D000DACFE6FFE1CFD9FFE2CFDAFF89E9066A5D
:1041E0001200F3DF068001D0F0DF01AEFEEF20F019
:1041F000006C011EE86A012206B0067E03AE06EFDF
:1042000021F0026C031EE86A0322067EC3EC21F053
:1042100003BE28EF21F006AE08D0026C031EE86A48
:104220000322046C051EE86A052206B006D084EB62
:1042300000F085EB01F006A004D082EB00F083EBE8
:1042400001F0E552E5CFDAFFE7CFD9FF45E9000CF1
:1042500006BE0DEF21F0E9DFFF0C44E8D9CFE6FF01
:10426000DACFE6FFE1CFD9FFE2CFDAFF8AE980EBD0
:1042700004F081EB05F082EB06F002500402F450EA
:10428000016EF350006E0350076E0502F450036E8A
:10429000F350026E07500402F3500126F45002223C
:1042A000E86A032206500502F3500126F450022268
:1042B000E86A0322E552E5CFDAFFE7CFD9FF46E906
:1042C000000C44E8D9CFE6FFDACFE6FFE1CFD9FF13
:1042D000E2CFDAFF8EE980EB08F081EB09F082EBA8
:1042E0000AF083EB0BF004500802F350006EF45018
:1042F000016E04500902F3500126000EF420026EF4
:1043000004500A02F3500226000EF420036E0450FB
:104310000B02F350032605500802F3500126F45017
:104320000222000E032205500902F3500226F45027
:10433000032205500A02F350032606500802F350E8
:104340000226F450032206500902F35003260750B8
:104350000802F3500326E552E5CFDAFFE7CFD9FF95
:1043600048E9000C43E8D9CFE6FFDACFE6FFE1CF1A
:10437000D9FFE2CFDAFF89E9066A1200F3DF06808F
:1043800003D0F0DF01D00682056A046A100EE76EE2
:10439000D89002360336043605360050045C0150CE
:1043A000055805E30050045E0150055A022AE72E25
:1043B000F0D706B2120006B006D084EB00F085EB11
:1043C00001F006A004D082EB00F083EB01F0E5528F
:0C43D000E5CFDAFFE7CFD9FF45E9120086
:0443DC00D9CFE6FF50
:1043E000E1CFD9FF88E942E8010E0616060E062441
:1043F0000101E838F00B206F050E2025A9D8010136
:10440000226F0F0E2215216F2151080802E2080EBB
:10441000216F02EBE9FF03EBEAFF21C1EFFF020E80
:10442000202596D8096E09A628D001012029A7D8F1
:1044300076D884D8FEE10950E00BE838E840070B55
:10444000AAD8A4D8020EE76E79D8FEE10914A3D841
:1044500084D8030EA4D881D8040EA1D8010122ADBE
:104460000AD0065003E0E66A020E02D0E66A010EA8
:104470007FD8010E43D0030E1AD00101202968D83D
:104480000101136F4CD85AD8FEE10950E00BE8380F
:10449000E84081D809A80AD0065003E0E66A020E77
:1044A00002D0E66A010E64D8020E28D0040E086E0F
:1044B000060E0101202702EBE9FF03EBEAFFEFCF35
:1044C00021F101012151210700090FE02051202B8A
:1044D0003FD8E66E00EBE9FF01EBEAFF002A000E91
:1044E0000122E552E750EF6EECD7065003E0E66A92
:1044F000020E02D0E66A010E3BD8085043E9E7CF2E
:10450000D9FF1200146B156B166B40D81351EE12C5
:104510001451EE121551EE121651EE121200146BD8
:10452000156B166B33D8EE6E14C1EEFF15C1EEFF9E
:1045300016C1EEFF2BD8030EE76E1200D890EF36AF
:10454000010EEB36020EEB36030EEB36E7061200D9
:10455000E66E1AEC27F041E9120018D8EF50EE6A27
:10456000EFCFF4FFEE6EEF50F4CFEEFFEF6E1200E0
:10457000E66E2C0EE66EF8EC26F043E91200E8DF5A
:104580000101216FE8CF13F10101120004EBE9FFF3
:1045900005EBEAFF12000101136F82EF22F0010127
:0845A0002025EDDF82EF22F07F
:0845A8006DA60FD802D06DB61C
:1045B00013D801011C0508E16DBA06D0686A696A62
:1045C00069806988020E1C6F12006D6A696A6D86C7
:1045D0000101010E1C6F12006D6A696A01011C6BFA
:1045E0001200ECEF22F001011C5101E145D06850AE
:1045F000040B04E06950040B01E047D86DB23CD0D5
:104600006850010B04E06950010B01E06BD8685061
:10461000100B04E06950100B01E02FD86850400BDC
:1046200004E06950400B01E049D86850200B04E0D9
:104630006950200B01E044D86850020B04E0695037
:10464000020B01E04DD8030E01011C5D01E214D004
:104650000001FD6B040EFD5D0FE26850080B0BE0DE
:104660006950080B08E03DEC11F0000901E1689683
:104670000001FD2BEFD700D01200698468986D828D
:10468000A19AA08A0300A09A12006D92699468A46E
:1046900002D06894FCD7120001011DA10ED06D92CA
:1046A0006D840001080EFE6F070EFF6FFE07000EFF
:1046B000FF5BFE51FF11FAE16D941200689C12003D
:1046C00070A00CD0800E0401005D07E1840E04018F
:1046D000045D03E104018C0E006F7090689A120073
:1046E0006A6A12006A6A686A9F0E6B6E7B0E696E58
:1046F0006E6A0F0EE66E710EE66E0F0EE66E18D83D
:1047000043E9160E706E68A608D068960000000097
:104710000000000000000000F6D76D98A0EC12F039
:1047200001011D9101011E6B0101030E1C6F12009E
:10473000D9CFE6FFE1CFD9FF84E901EBE9FF02EB36
:10474000EAFF005003E0EE6A0006FBD741E9E7CF3D
:04475000D9FF12007B
:0C475400FE0EE3CFE9FFFF0EE3CFEAFF0B
:10476000EFCFF3FF030EEF26F36EE926000EEA22E9
:10477000040EEDCFEBFFF32EFCD7680EEC6E6A0E45
:10478000EC6EF10EEC6EFD0EEB501200FE0EE3CF60
:10479000E9FFFF0EE3CFEAFFEFCFF3FFF3CFF4FF24
:1047A000F42AF4CFEEFFE86AEE24F32EFDD7EF6E85
:1047B000F4501200FE0EE3CFE9FFFF0EE3CFEAFF55
:1047C000EFCFF3FF030EF35E0AE009E6F3CFF4FF49
:1047D000F3CFEEFF030EEBCFEEFFF32EFCD7F4503A
:1047E0001200FE0EE3CFE9FFFF0EE3CFEAFFEFCFAB
:1047F000F3FFF306F3CFF4FFF3CFEEFFE86AEE2406
:10480000F32EFDD7EF18D8B4F4501200D9CFE6FF3D
:10481000DACFE6FFFC0EE3CFE9FFFD0EE3CFEAFFC0
:10482000F90EE3CFF4FFEFCFF3FFEF50E926000ED0
:10483000EA22030EF4B0E82AD96EE82AEDCFEBFFA6
:10484000F32EFCD7EFCFF3FFD950EF26FA0EE3CFCC
:10485000D9FFFB0EE3CFDAFFE86AF4A0F350DE10D5
:10486000EC6EDECFECFFDECFECFFF4B0F3CFECFF6D
:10487000E552E7CFDAFFE552E7CFD9FFF4B002D037
:10488000FD0E01D0FC0EEB501200D9CFE6FFFD0E5D
:10489000E3CFE9FFFE0EE3CFEAFFEFCFF3FF010E18
:1048A000EB503F0B030ED8B4E82AD96EF35E0AE052
:1048B00009E6F3CFF4FFF3CFEEFFD950EBCFEEFFD5
:0E48C000F32EFCD7E552E7CFD9FFF4501200DB
:0248CE008984DB
:1048D000C80E04D88994120089941200E84E05D0BD
:1048E00000D000D000D000D0F9D7000000D000D018
:1048F00000D01200E9CFE6FFEACFE6FFFC0EE3CFDF
:10490000E9FFFD0EE3CFEAFF43E8D9CFE6FFDACFB8
:10491000E6FFE1CFD9FFE2CFDAFF87E9EE50026E82
:1049200002520FE00EE648D8000909E0D0DFEE5051
:10493000046E16D8000903E0022EF9D702D0FF0E4C
:1049400002D0CADF010EE552E5CFDAFFE7CFD9FF8B
:1049500043E9E552E7CFEAFFE552E7CFE9FF12006E
:10496000080E036E03B01AD0899404AE02D03F0E35
:1049700002D01F0E0000B2DF04AE05D0FF0ECF6ED6
:104980009F0ECE6E05D0FF0ECF6ECF0ECE6E000006
:104990009E909EB00BD080B20ED0FBD7898404AE1F
:1049A00002D0400E02D0800E000098DF034E02D0ED
:1049B0000446D8D7010C000CDB0ED76E600ED66E05
:1049C000F29480A203D0F2B414D0FBD7FE0ECF6EC7
:1049D000780ECE6E9E9080B2F6D79EA0FCD7FF0ECA
:1049E000CF6EC50ECE6E9E9080B202D09EA0FCD738
:0449F000010C000CAA
:0C49F4003F004F4B00454C4D3332372044
:104A000076312E3120636F6D70617469626C650060
:104A10004F4244444941472E4E45542076342E316E
:104A20003420627920416C6578205369646F726527
:104A30006E6B6F0044415441204552524F52003C2E
:104A400044415441204552524F52004E4F20444160
:104A50005441004552524F52004642204552524F57
:104A60005200425553204255535900425553204558
:104A700052524F5200554E41424C4520544F204314
:104A80004F4E4E4543540050726F6772616D204522
:104A900072726F720031322E305600FB2FF62FF1FA
:104AA0002FED2FE82FE32FDE2FDA2FD52FD02FCBAE
:104AB0002FC62FC12FBC2FB72FB22FAD2FA82FA3DA
:034AC0002F9E2FF7
:0D4AC3001201000202000008D8040A0000E1
:104AD00000010203010902430002010080320904BF
:104AE000000001020201000524001001042402025A
:104AF00005240600010524010001070582030800C2
:104B00000209040100020A00000007050302400038
:104B100000070583024000000403090418034F0046
:104B20006200640044006900610067002E004E00CE
:104B3000650074001A034F00420044003200200058
:104B4000410064006100700074006500720016038B
:104B500031003700340031003500320032003400BB
:104B600035003500D54AD54A184B1C4B344B4E4BBB
:024B7000E62538
:0E4B72000F0EC16E880E8A6E936A896A2B0E32
:104B80009216010EB46E8B6A860E946EF29EF29CA3
:104B9000D56EF28AB50ECD6E9D80CB68050ECA6EBD
:104BA0009D80010EB46E1200D9CFE6FFE1CFD9FF90
:104BB00081E942E8D950010FE66EDACFE6FF91ECC9
:104BC0001DF042E9120E025C0AE11F0E0114010100
:104BD000136F040E135D03E20001008902D000018F
:104BE000009943E9E7CFD9FF1200140E6F6E01015F
:104BF0001C6B01011D6B01011E6BBBDFCEEC1AF0BB
:104C0000D9EC08F0D4EF25F0F0DFD1EC1AF050EC3D
:0A4C10001AF028EC1AF0F9D7120090
:064C1A002A0EF66E000EEA
:104C2000F76E000EF86E01010900F550056F0900DE
:104C3000F550066F03E1056701D03DD00900F5503E
:104C4000006F0900F550016F0900F550026F09006F
:104C50000900F550E96E0900F550EA6E09000900F7
:104C60000900F550036F0900F550046F09000900B1
:104C7000F6CF07F1F7CF08F1F8CF09F100C1F6FF41
:104C800001C1F7FF02C1F8FF0101035302E1045320
:104C900007E00900F550EE6E0307F8E20407F9D7C4
:104CA00007C1F6FF08C1F7FF09C1F8FF01010507B9
:084CB000000E065BBFD71200E5
:084CB800D9CFE6FFE1CFD9FFDF
:104CC00084E9AC6AAB6A02A005D0AC8802A404D027
:104CD000AC8E02D002B8AC8402A202D0AC8CAB8CF9
:104CE00002A602D0AB8801D0AB8A02AC02D09D8A6A
:104CF00001D09D9A02AE02D09D8801D09D9800EB14
:104D0000AFFF010101EB13F1146B13C1B0FFAC8ACB
:0A4D1000AB8E41E9E7CFD9FF120096
:064D1A00D9CFE6FFE1CF56
:104D2000D9FF82E9005005E1080EE66EE66E300E0E
:104D30000ED0000405E1080EE66EE66E400E07D0C8
:104D4000020E005C09E1080EE66EE66E500EE66E9D
:104D5000F8EC26F043E902D0FF0E01D0000E41E945
:064D6000E7CFD9FF1200AD
:0A4D6600D9CFE6FFE1CFD9FF81E9C4
:104D700042E8026A8290016A070E015C0BE28280BF
:104D80008050200B01E0010E0226029E0246829016
:104D9000012AF2D782808050200B01E0010E02260A
:0C4DA0008290025043E9E7CFD9FF1200D7
:044DAC00D9CFE6FF76
:104DB000E1CFD9FF82E941E88290026A080E025CE5
:104DC00012E28290005002EBF3FF025204E0D8900E
:104DD000E836F306FCE1800B02E0818C01D0819C77
:104DE0008280022AEBD7000E42E9E7CFD9FF1200FA
:104DF000D9CFE6FFE1CFD9FF84E922EC28F0050EF8
:104E0000E66E13D8FCE102EBE6FF0FD8FCE101EB04
:104E1000E6FF0BD8FCE100EBE6FF07D8FCE124EC51
:104E200028F041E9E7CFD9FF1200D6EC26F041E99E
:044E30000009120063
:0C4E3400D9CFE6FFE1CFD9FF82E941E8C9
:104E400022EC28F0030EE66ED6EC26F041E90009CC
:104E5000F9E100EBE6FFD6EC26F041E90009F9E1C3
:104E6000B3EC26F0026E24EC28F0025042E9E7CFC2
:044E7000D9FF120054
:0C4E7400D9CFE6FFE1CFD9FF83E922ECA3
:104E800028F0020EE66E0FD8FCE101EBE6FF0BD82E
:104E9000FCE100EBE6FF07D8FCE124EC28F041E957
:104EA000E7CFD9FF1200D6EC26F041E90009120045
:104EB000FF0EE3500101296FEE0E02D0F20E00004A
:104EC000E76EE72E61EF27F00C0E0101286FE76A0D
:104ED000E72E68EF27F0282F67EF27F00101292F31
:064EE0005EEF27F0120056
:0A4EE600D9CFE6FFE1CFD9FF81E943
:104EF00041E822EC28F0A00EE66ED6EC26F041E95F
:104F0000B3EC26F0016E24EC28F0015042E9E7CF23
:044F1000D9FF1200B3
:0C4F1400D9CFE6FFE1CFD9FF81E942E8E8
:104F2000CE50016ECF50026E01EBF3FF02EBF4FFA7
:084F300043E9E7CFD9FF1200AD
:084F3800D9CFE6FFE1CFD9FF5C
:104F400083E942E880EB03F081EB04F004EBD7FF48
:0C4F500003EBD6FF43E9E7CFD9FF1200C6
:044F5C00D9CFE6FFC4
:104F6000E1CFD9FF82E900EBE6FFE00EE66E0F0E1F
:104F7000E66EF8EC26F043E941E9E7CFD9FF1200ED
:104F8000D9CFE6FFE1CFD9FF81E941E80E0EE66E09
:104F90001AEC27F041E9016EE00E011442E9E7CF77
:044FA000D9FF120023
:0C4FA400FF0EE3500101296F480E01D000
:104FB0004C0EE76EE72EFED7E76AE72EFED7292FC5
:044FC000F7D712000D
:0C4FC40013EE00F023EE00F0F86A0DEC94
:0E4FD00026F028EC28F004EC26F0FBD71200A7
:024FDE000201CE
:104FE00000000000000030313233343536373839B4
:064FF00041424344454626
:0A4FF600018102010000013E425556
:0D50000053494E49543A20002E004F4B00FA
:02500E0022EC92
:1050100028F0C00EE66ED6EC26F041E90009F9E171
:0450200024EF28F061
:0C502400D9CFE6FFE1CFD9FF84E941E9D4
:06503000E7CFD9FF1200DA
:0A50360000EE00F00F0EEE6AEA62D1
:04504000FDD7120086
:08504400819E1200818E120012
:02504C00486BAF
:02504E00416BB4
:0250500012004C
:0250520000005C
:0C505400F331E531D731CC31B4319D315E
:1050600084316B3152313931F33125311131003115
:10507000E230C530A630873068304930473045309F
:10508000433041303F303D303B30393037303530C0
:10509000473032302F302C3029302630233020302A
:0450A0001D301A3075
:020000040030CA
:0100000024DB
:010001000EF0
:010002003FBE
:010003001EDE
:0100040000FB
:01000500807A
:01000600C138
:0100070000F8
:010008000FE8
:01000900C036
:01000A000FE6
:01000B00E014
:01000C000FE4
:01000D0040B2
:00000001FF
